:030000000219FDE5
:03000B000200A848
:03002B000201636C
:03005B000202EDB1
:030073000202D3B3
:1000800002030406080C10182030406080040608A3
:100090000C10182030406080A0C000070F1F3F05E3
:1000A000050D050305030302C2AFC0D0C0E0206206
:1000B00017E5256002E473E525F4F58A758B00D217
:1000C00062D0E0D0D0D2AF3285268AC262E526F473
:1000D0006035306803207210758B00D0E0D0D0D22C
:1000E00092D291D290D2AF32D292D291D290206E4F
:1000F0000C2066097405D5E0FDE57E4290758B0005
:10010000D0E0D0D0D2AF32758A00C28DD26201FD6C
:1001100001B7306805206602C29201B73068052039
:100120006602C29101B7306805206602C29001B72D
:10013000C29530680A2066077403D5E0FDC29201BB
:10014000B7C29430680A2066077403D5E0FDC291F7
:1001500001B7C29330680A2066077403D5E0FDC278
:100160009001B7C2AFC2AD53E6EFC0D0C0E0D2D36A
:10017000D2AFC2CEE52A6007207449152A21C4787F
:1001800000790020742EE580307E01F430E702789B
:10019000FF53DACF207E0343DA20307E0343DA10A8
:1001A000C2D8C271E580307E01F430E70279FFC326
:1001B000E89970CB306103752A18207403752A18EA
:1001C000885FD27020740DE52B6004152B21D44379
:1001D000DA01C2D82070024136A85F206102C270E5
:1001E000207431C3E894F0400374F0F8E8C4540F6D
:1001F00028F87984B703024114C313C3138721205D
:100200000802C313200A06C3C898F8411428F850FE
:100210000374FFF8C3E895685003E568F88822E5A1
:100220002D54066011E533C313C31324062522F5AC
:100230002250037522FF852224A824C3E524956457
:100240004002A8648825E5697002417AC3E8AA697A
:100250009A5003E8FAE4F9EAC333FBE56BF45B294F
:10026000400D256AF8E56A6002156A400B417A0A7A
:10027000C3E56A9A5002056A78FF8826C26EC3E514
:100280002694F84002D26EC3E52594404002D26421
:1002900020CF0AD0E0D0D043E610D2AD32C2CF0595
:1002A0003A7801E52A6005307402152AC3E55F94A7
:1002B00001400575620041C9756300756C00E56217
:1002C0002401F56250037562FFD0E0D0D043E61000
:1002D000D2AD32C2AFC0D053E67FC2607591008507
:1002E0005694855795759104D0D0D2AF32C2AF5392
:1002F000E6EFC2ADC0D0C0E0C0F0D2D3D2AFA8FB11
:10030000A9FCC2D8307102615453DACF207E034376
:10031000DA10307E0343DA20D271E580307E01F4BA
:1003200020E702612B88278928A17B53DACF207E22
:100330000343DA20307E0343DA10C2D8C27130742E
:1003400002A1677800E580307E01F430E702A16702
:10035000885FA14F53DACF207E0343DA20307E033B
:1003600043DA10C271206102812D53DACF207E035F
:1003700043DA10307E0343DA20C2D8D271885A891A
:100380005BC3E89558F8E99559F97B007E087A0037
:10039000C3E8948CE994005005755E00811F8821A4
:1003A00078A2E6A8216055C3E894C8E994005008F3
:1003B000E4D2E4FB7A0A61FAC3E89468E994015054
:1003C00008E4D2E3FB7A0F61FAC3E894D0E994021F
:1003D0005008E4D2E2FB7A1E61FAC3E894A0E994E3
:1003E000055008E4D2E1FB7A3C61FAC3E89498E94D
:1003F00094085008E4D2E0FB7A787E00C3E8955C6C
:10040000FCE9955DFD30E70AECF42401FCEDF434E1
:1004100000FD755E00C3EC9AED9E5003755E018889
:100420005C895D855A58855B597802A14FC3E89570
:1004300027F8E99528F9307C02A133307B02A133FB
:10044000307A02A12C2075028150E9FDE8FC816F11
:10045000E9C313F9E813F8307902A12CE9C313F9C1
:10046000E813F8307802A12CE9C313FDE813FC204F
:0E0470006126C3EC941CED940240028186EDDF
:10047E007018C3EC94C850120529C3E529940A508C
:10048E0002A167755F00D270A167E5296002152988
:10049E007888E6F97400207F087896B90302789E72
:1004AE00E624FAFEE43400FFC3EC9EFCED9FFD92C1
:1004BE0008B90310A2085007207609D27681D230EF
:1004CE007602C276A2085016B9030DECF42401FC94
:1004DE00EDF43400FD0204EC78007900A133B90389
:1004EE0015EC33FCED33FDC3EC940AFCED9400FDEA
:1004FE0050047C007D00C3EC94FFED940040067820
:10050E00FF7900A133EC8575F0A4C5F0A2F733F89E
:10051E007900400302054F78FF790002054FE9C3C9
:10052E0013F9E813F8307C0EE9600278FFC3E81384
:10053E0038F8E43400F9C3E894FFE99400400278F7
:10054E00FF885FD270206102A167741FF4552F4B94
:10055E00F52FC274EB7002D274752A1830740375BD
:10056E002A0A306102A17B20740353DAFE20740341
:10057E00752B06D0F0D0E0D0D0D2AD43E610327954
:10058E00010205AB79030205AB790A0205AB791EB0
:10059E000205AB79640205AB79C80205AB7817E4A6
:1005AE00D5E0FDD8FAD9F6227A147B780205D27AF4
:1005BE00107B8C0205D27A0D7BB40205D27A0B7BAE
:1005CE00C80205D27902B27DE4C294D5E0FDC29193
:1005DE00D5E0FDD291D5E0FDD294D5E0FDC292E5F5
:1005EE0076D5E0FDD2927496D5E0FDD9D9EAF8D54C
:1005FE00E0FDD8FBDBCEC29422C37C007D0075F0FB
:10060E000005F0EA33FAEB33FB50F6EB13FBEA137B
:10061E00FAC3E9FFE8FEE89AF8E99BF95004EFF90E
:10062E00EEF8B3EC33FCED33FDD5F0DFEDF9ECF87D
:10063E0022E889F08A20D2D4F8A9F07B0030F70B9B
:10064E007BFFF42401F8E9F43400F9E88520F0A4E6
:10065E00ADF0F8E98520F0A4AFF0FEED2EF97400B0
:10066E003FFA7C04C3EA13FAE913F9E813F8DCF451
:10067E008BF030F70AE8F42401F8E9F43400F9E8D5
:10068E0089F0C2D4F8A9F02222C3E54113F9E5405E
:10069E0013F8C3E54598F8E54699F9500CC3E8946C
:1006AE0080E994FF40160206CEC3E8947FE99400D9
:1006BE0050030206CE787F79000206CE788079FF4D
:1006CE00884A894B22E54A2547F8E54B3548F98596
:1006DE004B20E4300701F43549FA30E709C3EA94B8
:1006EE00F0401502070CC3EA940F500302070C7872
:1006FE00FF79FF7A0F02070C780079007AF0C3E5D4
:10070E00249564500AC374019524500B02072AE500
:10071E004B20E70E02072AE54B30E706884789484B
:10072E008A492278A4E6FAC3E54A33F8E54B33F951
:10073E00D13FE930E70BC3E89480E994FF4013E121
:10074E0064C3E8947FE994005002E164787F7900F5
:10075E00E164788079FFE820E715C3E52398F84037
:10076E0009C3E89401400302078B780102078BE866
:10077E00F424012523F8400302078B78FF884C22CE
:10078E0078A5E6FAA848A949D13FE930E70CC3E8B5
:10079E009401E994FF40160207BFC3E894FFE99461
:1007AE000050030207BF78FF79000207BF78017976
:1007BE00FFE920E715C3E54C98F84009C3E894011A
:1007CE0040030207E678010207E6E8F42401254C0F
:1007DE00F840030207E678FF88242278FFC26420DF
:1007EE00693D206A12D264C3E541940A4009C3E50B
:1007FE002594405002C26479A1E76023E541601F51
:10080E0074FF8541F0848539F0306A0375F005A4D4
:10081E00F8C5F0600278FFC3E895675002A86788B4
:10082E006622C3E5409440E5419401E56650031409
:10083E000141046002F566220208492275E8902201
:10084E007883E6FFE5E820ECF7A8BDA9BE0573C3E3
:10085E00E57394084052757300E9FA79A0E7604495
:0E086E00EA7007E574601B020884C3E8957405
:10087C006010E5745006600C140208900460F902D4
:10088C000890E574F574C3946D401B7564C0C394F3
:10089C00044013756480C39404400B756440C39486
:1008AC0004400375640075BB0622E564F460020520
:1008BC0064E573B4070375BB1022743279A687F014
:1008CC00A4C5F0A2F733F8C3E895644002A8648885
:1008DC00228824882588268867227540007541F077
:1008EC0022C2AF75C820A8CCA9CDAA3A30CF010A34
:1008FC0075C824D2AFAB3BAC3C883B893CC3E89B6E
:10090C00F8E99C206908F93067024102215FAD3D8E
:10091C008A3DF9EA9DFA600478FF79FFAE3EAF3F5D
:10092C008B3E8C3FC3EC9FFCC3E99CF542A83BA9D2
:10093C003CC3E89EF8E99FF9C3E54113FBE540137E
:10094C00FAE82AF540E93BF54150067540FF754140
:10095C00FF21A9AA40AB41AC40AD417E047F02C34C
:10096C00EB940440021E1FC3EB940840021E1FC3ED
:10097C00ED13FDEC13FCDEF7C3EA9CFAEB9DFBEFE9
:10098C006009C3E913F9E813F8DFF7EA28FAEB3941
:10099C00FB8A408B4150067BFF8B408B41C3EB9411
:1009AC00025002D2673069047F0321D47892E6FFAB
:1009BC00C3E537948240110FC3E53794A040010F73
:1009CC00C3EF940640027F057E04E541C4540FF941
:1009DC00E541C454F0F8E540C4540F28F8C3E89E30
:1009EC00FAE99400FB4009C3EA9402EB940050042A
:1009FC007A02E4FB414EAA40AB41EBC4FEEAC4547C
:100A0C000F4EFCC3EA9CFAEB9400FBC3E813C31330
:100A1C00F8EA28FAEB3400FB8A408B41C3EB9402D2
:100A2C004002C2677804EBC4FE7B00EAC4540F4E4C
:100A3C00FAC3EA98FA4005C3940250027A027892FB
:100A4C00E6FF306002414E855256855357D26043C3
:100A5C00E680C3E49AF8E49BF930670241E8E8FACF
:100A6C00E9FBD3E913FDE813FC88528953C3EF94D7
:100A7C00036038EF20E00DE82CF8E93DF9ECFAEDD5
:100A8C00FB020AA3E828F8E939F9C3E82402F8E9DB
:100A9C003400F97AFE7BFFC3EF9403400E8A548B2B
:100AAC0055884E894F8C508D51611C885489558ABC
:100ABC004E8B4F8C508D51306920C3E533940340DD
:100ACC0019E542A2E713F8E555F4240138400B2050
:100ADC00E7087554FFF42401F555611CE8FAD3E8D6
:100AEC0013FC8852C3EF94036020EF20E007E82C3E
:100AFC00F8ECFA6108E8282402F87AFEC3EF9403B4
:100B0C0040088A54884E8C50611C88548A4E8C50F4
:100B1C00E56BC3335002646BF56B30600261267574
:100B2C003402D26043E680E52D54066026A840A925
:100B3C0041C3E913F9E813F8C2AF53E67F7591008E
:100B4C00C3E498F594E499F595759104D26043E665
:100B5C0080D2AF22D265754400752000306B0375CE
:100B6C002040020B7FD265754400752040306B032A
:100B7C00752000D2AF7801206722E52D5406600263
:100B8C00C265C3E54194054013780294054008788A
:100B9C0003940540027806306902780A206019E552
:100BAC0044601530690AC3E53394034003D5340619
:100BBC00D2AFD26C8151712ED2AF0000C2AF206780
:100BCC0026E541C3FB940F40027B0FEB24053073E9
:100BDC000123306A02742820620123F930690279FA
:100BEC0082E58BC39940B50544E59BF45440B52090
:100BFC0002813B30690A08C3E8940A40010861A8E5
:100C0C00206502617FC26553E67F759100306710E5
:100C1C007594007595FE759104D26043E680617FF2
:100C2C00AE40AF41C3E49EF594E49FF5958122C399
:100C3C00E53394025002617F306502617FD80281F6
:100C4C004F61A8C26C53E67F75910085549485550D
:100C5C0095759104854E56854F57D26043E680D2E8
:0F0C6C00AFE52D54066008206A020533020C8B99
:100C7B00306C0D206B0A2065071581158102150854
:100C8B002278003064053065027801E53775F0078E
:100C9B00A4F9E5F028F5F0E9A2F013A2F113A2F202
:100CAB0013F537C394785003753778C3E537953808
:100CBB004008D266D292D291D29030600281C58523
:100CCB005056855157D26043E68022207D11C2AF2A
:100CDB00754302C294D295D2AF759F11020EA5C275
:100CEB00AF754302C294D293D2AF759F11020EA57A
:100CFB00307243207D20C2AF754303900141757E56
:100D0B0010D290C293306204C291A119D294D2AF87
:100D1B00759F01020EA5C2AF754303900141757E0D
:100D2B0010D292C295306204C291A139D294D2AF43
:100D3B00759F21020EA5207D17C2AF75430390014D
:100D4B001CD290306202C291D2AF759F01020EA5E8
:100D5B00C2AF75430390011CD292306202C291D292
:100D6B00AF759F21020EA5207D11C2AF754304C242
:100D7B0095D293D2AF759F21020EA5C2AF754304D6
:100D8B00C293D295D2AF759F01020EA5307243204C
:100D9B007D20C2AF754305900130757E20D291C284
:100DAB0094306204C292A1B5D295D2AF759F110255
:100DBB000EA5C2AF754305900152757E08D291C244
:100DCB0094306204C290A1D5D293D2AF759F110219
:100DDB000EA5207D17C2AF754305900112D291303D
:100DEB006202C292D2AF759F11020EA5C2AF7543BC
:100DFB0005900126D2913062EBC290D2AF759F1154
:100E0B00020EA5207D11C2AF754306C293D294D2B8
:100E1B00AF759F01020EA5C2AF754306C295D29462
:100E2B00D2AF759F21020EA5307242207D20C2AF3A
:100E3B00754301900152757E08D292C295306204BF
:100E4B00C290C151D293D2AF759F21020EA5C2AFF2
:100E5B00754301900130757E20D290C293306204AD
:100E6B00C292C171D295D2AF759F01C1A5207D16DB
:100E7B00C2AF754301900126D292306202C290D26A
:100E8B00AF759F21C1A5C2AF754301900112D290DE
:100E9B00306202C292D2AF759F01C26622900110DE
:100EAB00757E00D292D291D290C295C294C293C257
:100EBB006222788076FF0876FF0876FF0876FF08B7
:100ECB00760308760408760A087603087601087616
:100EDB0001788C76010876FF0876FF0876FF087696
:100EEB00FF0876FF0876030876FF0876FF0876FF83
:100EFB000876250876D00876FA0876FA087604087C
:100F0B0076FF08760108760008767A0876FF087671
:100F1B0001087601087600087603227887E6FFC27F
:100F2B0072BF0302D2727888E6C394036008C27D55
:100F3B00E630E102D27DC27E7889E630E102D27ED4
:100F4B00C3EF94026008758E01D273020F5E758E2B
:100F5B0000C273227880E6149000809378A4F67810
:100F6B0081E6149000809378A5F67886E6149000BD
:100F7B008D9378A6F6789CE67538FF75390CB4021C
:100F8B00067538A075390AB40306753882753905AC
:100F9B0078A3E61490009A93F569D1A8222278964B
:100FAB00E6FA7897E6FB7888E6B40305C3EB940E74
:100FBB00FB307F047A007BFFC3EB9AFCC394825017
:100FCB00027C827575000575EC8575F0A4C3E5F0A0
:100FDB00947D40F222D27FF1A912059C7A007B000E
:100FEB007C10120592E55F2AFA74003BFBDCF37C64
:100FFB0004C3EB13FBEA13FADCF7FEC27F120FA953
:10100B0022E5EF20E6037520000520903FFFE52049
:10101B00146006901DFF1460009304600375EF12BB
:10102B0053D9BF7581C043FF8012058D75EF024305
:10103B00B203E5B3240420E70DF521E5E320E00638
:10104B008521B343E301120EA87580FF75A40075CB
:10105B00F19075D47F75900775A53F75F23F75D5E7
:0F106B000075A60175E241E4F8F6D8FD756B013A
:10107A00120EBD12154A78988676753001C2AF12E3
:10108A0005A61205B612059C1205BD12059C12058D
:10109A00C412059C1216631205A61205A61205A112
:1010AA00C2AF78FA79FA308707D9FBD8F7021C0061
:1010BA00120F26120F5F120FA8120FA978988676C0
:1010CA00120EA875885075891275C8247591047511
:1010DA00D84075A82275B80275E690759B80759DF3
:1010EA000075D10E75BC5875BB0675BA1175E880C6
:1010FA0012058DD2AF12084653DACF207E0343DAA7
:10110A0020307E0343DA1043DA01C2D8C2711205D5
:10111A00A6D2617B037A0CE55E70077A0CDB0302C8
:10112A0010AA12059C2070030210AAC270E55FC3C0
:10113A00940240E1E52F541F856160F561B560D5E1
:10114A00DAD5C26153DACF207E0343DA20307E0338
:10115A0043DA10C2D8C27178A2E67008D274E52FB9
:10116A0054E0F52FC2757529001205A1307409C320
:10117A00E529940A4002D275120592780230740267
:10118A007800C3E55F9840F0C2AF1205B61205B603
:10119A001205B6D2AF1205A6754D007888E6B403DB
:1011AA0002418A120592788CE6C394015003021216
:1011BA008AE530C39401500302128A207435C3E5CC
:1011CA005F94FF500302128AC2AF1205CBD2AF124C
:1011DA0005A1C3E55F940150EFC2AF1205B612052F
:1011EA00971205B6D2AF1205A1C3E55F94FF40E995
:1011FA000216E87F05D27F120FA91205A1C2AFC25B
:10120A007F120FA9AE5FC3E55F947FD2AF407B1216
:10121A00058DC2AF1205CBD2AFDFDA120FE0C3EEF3
:10122A0094057897F61205A612158C12166B7F0A8A
:10123A00D27F120FA91205A1C2AFC27F120FA9AEA7
:10124A005FC3E55F947FD2AF50E412058DC2AF123F
:10125A0005B61205971205B6D2AFDFD4120FE0EE2B
:10126A0024057896F61205A612158C12169A1205FE
:10127A00A1120FA9C3E55F94FF500221C50216E827
:10128A00C3E55F954D4003855F4D1205A17801794D
:10129A0088E7B403027805C3E55F98400221A5C236
:1012AA00AF1205CB1205CB1205CBD2AF1205A6752C
:1012BA003000E4F531F5320531E531F470390532A3
:1012CA00789AE67819146012783214600D787D14D1
:1012DA00600878FA146003753200C3E53298401743
:1012EA0015327531B478998676C2AF1205CBD2AF72
:1012FA00789886761205A1120597E52A700530744A
:10130A000201AA78012074027806C3E55F9840A713
:10131A007888E6C3940360031205A1E52A700302E4
:10132A0010AAC2AF120EA8E4F522F523F524F5257A
:10133A00F526F56AD2AF7885E6C333F568E4F54554
:10134A00F546F547F548F549F573F52CF52DF537CA
:10135A0075730875BB1012058D12084AE5E820EC72
:10136A00FBA8BDA9BEE97001F8887412084E75730E
:10137A000875BB107887E6FE7602120F267887EE8C
:10138A00F6C2AF7564FF1208C68522648522658598
:10139A002266D2AF752201752401752501752601D1
:1013AA0085636C756D017888E6B40307C27D307673
:1013BA0002D27DD268D269753300120E0E120E3334
:1013CA001208E61208ED1208E61208ED1208E60203
:1013DA0013E9C2AF120F26D2AF75730075BB06129E
:1013EA000B71120696120C8C120CD61208ED120B07
:1013FA0060306D031206972067031207E93067030E
:10140A00120830120C8C120CFB1208ED120B713000
:10141A006D031206D3120C8C120D721208ED120B08
:10142A0060306D03120731120C8C120D971208ED01
:10143A00120B71306D0312078E120C8C120E0E12E3
:10144A0008ED12084A120B60120C8C120E331208A5
:10145A004E1208ED306932206B2F85676485676507
:0E146A0085636C756D0179187A0CC3E53399B2
:10147800400CC269D26A8A357564FF021493C3E5C9
:101488005F940140030213E9021510306A1B206BB8
:1014980018E535147004C26A61DCF535C3E55F945C
:1014A8000140030213E9021510753600C3E562789E
:1014B80082985054307404E52A604D7888E6B40365
:1014C80017207D0520760781E030760281E0206BC9
:1014D80007D26B856764812878F0306B058567646F
:1014E8007820C3E54198500261E9306B1BC26BC29A
:1014F8007D307602D27DD26A75351285676461E9DE
:101508000536E55F6002A113753600C2AF120EA85A
:101518007887E6FE7602120F267887EEF6E4F52243
:10152800F523F524F525F526F568C268D2AF12052E
:101538008D120EA8307409C3E5369405400201AA3D
:1015480041BC901A0D78201215CEE520B45A0CA390
:101558001215CEE520B4A50302156C120EBD1215A6
:101568008C02158B901A0378807B0A1215CEA3087B
:10157800DBF9901A0F788C7B181215CEA308DBF9CB
:10158800901A2722C2AF12160D1215E7901A00748E
:101598000E1215D3A374041215D3A374141215D301
:1015A800901A0378807B0A1215D2A308DBF9901AE7
:1015B8000F788C7B181215D2A308DBF912162012AB
:1015C80015FE901A2722E493F622E6438F01538FE3
:1015D800FD75EF0275B7A575B7F1F0538FFE22437D
:1015E8008F02438F0175EF0275B7A575B7F1901A91
:1015F8000DF0538FFC22901A0D745AB1D3901A0E25
:1016080074A5B1D3227A3079D07820901A40B1CE1F
:10161800E520F709A3DAF7227A3079D0901A40E763
:10162800B1D309A3DAF922AB77A878BB0102798490
:10163800BB02027985BB03027986BB04027992BB9F
:1016480005027987BB060279A3BB0702799CBB0810
:10165800027988BB09027989E8F7227C051205A678
:10166800DCFB22C2AF1205B61205BD1205C4120575
:10167800CB1205971205B61205BD1205C41205CB8B
:101688001205971205B61205BD1205C41205CBD274
:10169800AF22C2AF1205CB1205C41205BD1205B6A2
:1016A8001205971205CB1205C41205BD1205B61214
:1016B80005971205CB1205C41205BD1205B6D2AFA7
:1016C80022AE77AF78C2AF1205B61205B61205B6CC
:1016D800120597DEF21205CB120597DFF8D2AF227A
:1016E800D16BD163D163757701757801757900D1B4
:1016F800C97C05AD5F1205A6C3ED955F70F5C3E51E
:101708005F9401400AC3E55F94FF4032021724D179
:101718002FB18CD16BC2AF75EF12D163DCD50579CF
:10172800C3E5799403500280C6D1630578E5771440
:1017380090009F93F808C3E57898500280AED16373
:10174800D1630577C3E577940A5002809C120EBDD9
:09175800B18CC2AF75EF12D16330
:0319FD0002100CC9
:101A00000E0414FFFFFFFF03040A0301015AA5019E
:101A1000FFFFFFFFFF03FFFFFF25D0FAFA04FF01DE
:081A2000007AFF01010003FF41
:101A400023454D41584E616E6F3230412320202096
:101A500023424C48454C4923463333302320202031
:101A60002020202020202020202020202020202076
:101C0000C2AFC2D353D9BF7581C043B20343FF8073
:101C1000752438752503B1C975EF0275E24043F1AB
:101C20008053A47F75D400D2877DFA780379E67C4F
:101C300010752200752300901DD67B0675249875BB
:101C400025013087028142208708D8FBD9F9DCF7CB
:101C500081B4308708D8FBD9F9DCF781B4B189E4C5
:101C600093A3C39A6004DDC381B4DBDBB17B600264
:101C7000812B7B08E493FAA3B15CDBF87A30B15C8A
:101C8000752200752300B17BEAFCEBFDC3ED94FEE9
:101C9000400EB17B8A278B28ED30E0048A828B834B
:101CA000B17B7AC270D8C3ED94FE601350CEBD00F4
:101CB00025EC60097520007521FF0200008100A855
:101CC00027A9280809D804D90281D3B17FEA89AAB3
:101CD000F281C50D81A0C3ED94035049EDA2E092BD
:101CE000007AC5C3E5829400E583941C50902000DF
:101CF00010438F02438F0175B7A575B7F1F030001F
:101D00001FA827A9280809438F01538FFDD804D99C
:101D100002A12089AAE275B7A575B7F1F0A3A10DBC
:101D2000538FFC817C7AC1BD030CE493A3FAB140CC
:101D3000DCF8B138817C817EAA22AB23B15CEBFA5E
:101D4000EA6222752608C3E52313F523E52213F57D
:101D50002250066323A0632201D526EAB1C9B1C986
:101D600075260AEAF4200102D287300102C287B147
:101D7000C9C3134002C201D526EB22B17FEAFB2082
:101D80008702A17F308702A184752608AE24AF2583
:101D9000C3EF13FFEE13FEB1CDB1C9C3EA13308711
:101DA000024480FA30E703632201C3E52313F523DD
:101DB000E52213F52250066323A0632201D526D91C
:101DC000E52265236523F52222AE24AF250E0FDE22
:101DD000FEDFFCD20122424C48656C693437316326
:041DE000F3300601D5
:00000001FF
